:020000040000FA
:0A0000000000AC2800000000000022
:04000A00003400348A
:02000E009C0153
:10001000B82130302C20B52130302C20B5213030A3
:100020002C20B52120302C20B221283022209C0108
:100030000C302220013022200630222008309C0083
:10004000B221080095000230A3001508F0392C20D9
:10005000950EA30B25280800860000001C078600CB
:10006000000000000000051600000000000005125E
:10007000A821080080303D28C0309D00A8219C01A7
:100080001D081E07222008309C0008009F00063033
:100090009E003C204C289F005520003E031908007C
:1000A00022209F0A0319A00A4C2820088A001F0852
:1000B0008200503449344334523441344434493456
:1000C0004F34003420347634203431342E343034FC
:1000D000333400344D3445344D344F345234493484
:1000E00053344534003449344E3449345434203484
:1000F0004F344B3421340034203420342034203425
:100100002034203446344D3400349E013A200030EF
:10011000A00059304B203C200030A00062304B2022
:1001200008009E013A200030A0006A304B20BE211A
:100130003A200030A00059304B2008009E013C209E
:100140000030A00073304B2008009E013C2000309E
:08015000A0007C304B200800E8
:080158008901831600308100CB
:10016000023085000730860083120430850010308D
:100170008B002329D321A130E0210D30E0218030F4
:10018000DD218030D7210030DA21D5210800D321AC
:100190006030DD211A08E0211B08E0210030D72162
:1001A0008030DA21D52108009E013C200D08031182
:1001B000003C0319EA280D08303E22200E08303E8C
:1001C00022200F08303E22202E3022201008303E00
:1001D0002220080020302220DE2819149B0FF1284D
:1001E0009A0A1B080311A43C031D3C291A08031199
:1001F000043C031D3C2903309A00D6309B003C2967
:100200001914013003109B02031807299A031B08D5
:100210000311D53C031D3C291A080311033C031D9F
:100220003C2904309A00A3309B003C29191C422928
:100230001A0888000030F4211B0888000130F421DE
:1002400019109120422907208520C12186183329C1
:10025000043088000030F421623088000130F4213D
:100260009E20861C3129BA200030EC219A000130F2
:10027000EC219B00A5201910C7204B215521D4202B
:10028000BB214229861CED28061D0029851C162944
:060290008B1063004229FF
:0A0296001A088F001B0890006B305F
:1002A00003109002031C8F03080000001130960019
:1002B0000430A2007B291930A3008C018D018E012E
:1002C00003108D0D03108E0D03188D0A03108F0D72
:1002D00003188E0A0310900D03188F0A0C0890075C
:1002E0008C0103100A300D02031C79298D000130A6
:1002F0008C00A30B602910080F39950016088400A4
:1003000015088000960AA20B5B29143096000E3067
:1003100097000330A20014088D001608840000081E
:1003200095000310950D1508950D950D1507950071
:1003300096031608840000088C0015088C02170824
:1003400084000C080F398000970AA20B8D29080041
:100350001F30AB29FA30A1000130A200CE290130B4
:10036000A200CC290230A200CC290530A200CC2961
:100370001E30A200CC29C830A200CC29FF30A20038
:10038000CC290430A400C6290830A400FF30A20004
:10039000CC21A40BC6290800FF30A100A10BCE2957
:0603A000A20BCC290800AD
:0A03A6008515080085110800A50068
:1003B0000130E229A5000230E229A5000430E2293B
:1003C000A5000830A20005110510A51B0514051590
:0803D000A50DA20BE3290800B2
:0803D8008900831608140818BF
:1003E000EF298312080808008900AF218316081539
:1003F00055308900AA30890088148818FD29831295
:020400000800F2
:02400E00F23F7F
:00000001FF
